:080000000C9446000C94000072
:100008000C9400000C9400000C9400000C94000068
:100018000C9400000C9400000C9400000C94000058
:100028000C9400000C9400000C9400000C94000048
:100038000C9400000C9400000C9467000C940000D1
:100048000C9400000C9400000C9400000C94000028
:100058000C9400000C9400000C9400000C94000018
:100068000C9400000C9400000C9400000C94000008
:100078000C9400000C9400000C9400000C940000F8
:100088000C940000F894EE27ECBBF1E0F5BFE5BF57
:10009800E0936C00F8E1F1BDE1BD8DE0A2E0BB2783
:1000A800ED938A95E9F780E090E1A0E0B1E0ED9367
:1000B8000197E9F78BBFEFEFEDBFE0E1EEBFC0E0DE
:1000C800D5E00C949400AA93BA93EA93FA93EFB705
:1000D800EA93A0E0B5E0ED91FD913196FE93EE93A1
:1000E80030D0D29710F4C09A11C02BD0A536E0E0DA
:1000F800BE0710F4C0980AC024D0A436E0E0BE07BA
:1001080029F4E0E0E0930005E0930105E2B7E76E2B
:10011800E2BFE991EFBFF991E991B991A9911895D9
:10012800E7E0E7BBC19AC29AE4E0E3BFE7EEE2BFCB
:10013800E1E0E7BF7894C19A09D0C19807D0FBCF16
:10014800FFCFA0910005B09101050895E4EFF1E01B
:10015800FA93EA930C94B000E991F991309639F04A
:1001680080EA9FE00197F1F7A8953197C9F70895BC
:00000001FF
